:100000000C942A000C94F1030C941A040C944700ED
:100010000C9447000C9447000C9466030C948A03DC
:100020000C9447000C9447000C9447000C94510228
:100030000C9482020C9447000C94D5040C94470055
:100040000C9447000C9447000C9447000C94470014
:100050000C94470011241FBECFE5D4E0DEBFCDBF16
:1000600010E0A0E6B0E0ECE6FDE002C005900D92E5
:10007000AC36B107D9F710E0ACE6B0E001C01D9294
:10008000A33BB107E1F70E9476000C94B4060C94F0
:100090000000982F813011F48FEF089580E09230A6
:1000A00009F481E00895982F813011F48FEF0895BD
:1000B00080E0923009F481E008951F93982F929583
:1000C0009F70182F1F709A301CF4892F805D02C01A
:1000D000892F895A1A3014F4105D01C0195A0E94F0
:1000E000D901812F0E94D9011F910895AF92BF922B
:1000F000CF92DF92EF92FF920F931F93CF93DF93F4
:1001000087B38F6087BB80E895E20E94A8010E94B8
:100110004C020E94B6020E94AE0380E090E00E9472
:10012000D80280E090E00E941F030E948D0485B3F6
:10013000806F85BBBC9A86EAE82E8EE0F82E789414
:1001400083B390E08073907004E0959587950A954D
:10015000E1F7813011F4AFEF04C0A0E0823009F480
:10016000A1E083B38295869586958370813011F4E2
:10017000EFEF04C0E0E0823009F4E1E0AF5FA330CC
:1001800018F000E010E00AC0BB27A7FDB095AA0F49
:10019000BB1FA05ABF4F0D911C911197EF5FE33029
:1001A00018F0C0E0D0E009C0FF27E7FDF095EE0FA2
:1001B000FF1FEA59FF4FC081D181C8010E94D802B8
:1001C000CE010E941F030115110509F0A1C020975F
:1001D00009F09EC0C7010197F1F788E00E949604DC
:1001E0008C0185E00E94960408521040081B190BF0
:1001F00089E00E949604EC0186E00E9496046E015C
:10020000C81AD90AE601CC0FDD1FCC0DDD1DD6952D
:10021000C795D695C795EC978AE00E9496046C0125
:1002200087E00E94960428ED3FEFC20ED31EC81A45
:10023000D90A580117FF02C0AA24BB24D7FF02C065
:10024000C0E0D0E0D7FE02C0CC24DD2490916C0049
:1002500080918700981721F5C50174E096958795E0
:100260007A95E1F70E945D008AE30E94D901CE01F0
:1002700064E0969587956A95E1F70E945D008AE3B0
:100280000E94D901C60154E0969587955A95E1F7E9
:100290000E945D008AE00E94D9018DE00E94D90190
:1002A0003DE2A31631E0B30654F460E09501220F5D
:1002B000331FCE018C0D9D1D821793070CF461E056
:1002C0008DE2C81681E0D8064CF410E0C601880F14
:1002D000991FCA0DDB1DC817D9070CF411E024E6DD
:1002E000A216B1040CF460E034E6C316D1040CF499
:1002F00010E081E00E94470482E0612F0E944704E1
:1003000060B3647080E00E94470460B368701CC0F2
:1003100060E0101611060CF461E081E00E944704D1
:1003200060E01C161D060CF461E082E00E944704A8
:10033000612F661F6627661F80E00E9447046E01DA
:100340006D2D661F6627661F83E00E944704F7CE67
:100350009C0140E050E084E0220F331F441F551FF2
:100360008A95D1F760EC71EE84EE90E00E949206DF
:100370002150304030BD29B90895F894E0916E00C5
:10038000F0E0E158FF4F808190916D00983021F4AA
:1003900090916E0090936D0090916E009F5F90938E
:1003A0006E0090916E00983010F010926E0078946C
:1003B0000895F894E0918700F0E0E159FF4F8083C1
:1003C000909187009F5F9093870090918700903174
:1003D00010F0109287002091870090916C002917EF
:1003E00019F490E190938700559A78940895CF93EB
:1003F000DF93EC0107C0909187009031E1F32196E3
:100400000E94D90188818823B1F7DF91CF910895A7
:10041000CF93DF93EC0106C0909187009031E1F318
:100420000E94D901FE01219684918823A9F7DF91CA
:10043000CF9108950F931F93CF93DF93EC018B011E
:1004400009C0809187008031E1F389910E94D90130
:100450000150104001151105A1F7DF91CF911F91B7
:100460000F9108950F931F93CF93DF93EC018B01AE
:100470000BC0809187008031E1F3FE0121968491C9
:100480000E94D901015010400115110591F7DF912B
:10049000CF911F910F91089588EB8AB908951AB8EA
:1004A00008951F920F920FB60F9211248F939F936E
:1004B000EF93FF938CB190916D009830D1F0E09163
:1004C0006D00F0E0E158FF4F808380916D008F5FF9
:1004D00080936D0080916D00883010F010926D0057
:1004E00090916D0080916E00981719F488E08093C8
:1004F0006D00FF91EF919F918F910F900FBE0F9024
:100500001F9018951F920F920FB60F9211248F9380
:100510009F93EF93FF9390916C00809187009817C1
:10052000D9F0E0916C00F0E0E159FF4F90818091AB
:100530008700803121F480916C0080938700809146
:100540006C008F5F80936C0080916C00803110F0A4
:1005500010926C009CB901C05598FF91EF919F914A
:100560008F910F900FBE0F901F9018958091B20041
:1005700082608093B20082B3806F82BB81B3806F50
:1005800081BB82EF8FBD81E08EBD89B789BF0895A1
:100590008FB7F89410928A001092890010928C0004
:1005A00010928B001BBC1ABC19BC18BC8FBF0895DD
:1005B00062E070E00E947F06862F972F22E0803055
:1005C0009207D4F42EEF813092071CF481E09EEF65
:1005D00002C097FF13C022273327281B390B309303
:1005E0008A0020938900969B04C0809188008270C5
:1005F00011C03BBD2ABD08958FEF91E090938A0012
:1006000080938900969B03C09BBD8ABD089580910D
:1006100088008160809388001BBC1ABC89B7806108
:1006200089BF08952091890030918A00220F331FDD
:10063000969903C0309521953F4FC901089562E016
:1006400070E00E947F06862F972F22E0803092076D
:10065000D4F42EEF813092071CF481E09EEF02C0AB
:1006600097FF13C022273327281B390B30938C00A8
:1006700020938B00979B03C039BD28BD08958091BE
:10068000880082600BC08FEF91E090938C00809384
:100690008B00979B0BC080918800817080938800AD
:1006A00019BC18BC89B7886089BF089599BD88BDF9
:1006B000089520918B0030918C00220F331F979B5F
:1006C00003C0309521953F4FC90108951F920F92A5
:1006D0000FB60F9211248F939F93859B14C082B302
:1006E0009091880090FD02C090E001C090E48F7B63
:1006F000892B82BB8091890090918A009BBD8ABD25
:1007000089B78F7E89BF9F918F910F900FBE0F90F9
:100710001F9018951F920F920FB60F9211248F936E
:100720009F93849B14C082B39091880091FD02C076
:1007300090E001C090E88F77892B82BB80918B007D
:1007400090918C0099BD88BD89B7877F89BF9F91A3
:100750008F910F900FBE0F901F90189585B78F60E7
:1007600085BF8BB7806C8BBF969A979808958FB78B
:10077000F89410928F0010928E00109291001092B7
:1007800090008FBF08958FB7F89410928F00109249
:100790008E008FBF08958FB7F89410929100109239
:1007A00090008FBF08959FB7F89420918E003091EC
:1007B0008F00882321F010928F0010928E009FBF2F
:1007C000C90108959FB7F89420919000309191004D
:1007D000882321F010929100109290009FBFC901D0
:1007E00008951F920F920FB60F9211248F939F932B
:1007F000969B0BC080918D008F5F80938D008091C0
:100800008E0090918F0001960AC080918D008150DA
:1008100080938D0080918E0090918F00019790932E
:100820008F0080938E009F918F910F900FBE0F903D
:100830001F9018951F920F920FB60F9211248F934D
:100840009F93979B0BC08091920081508093920060
:10085000809190009091910001970AC08091920040
:100860008F5F80939200809190009091910001960B
:1008700090939100809390009F918F910F900FBE65
:100880000F901F90189587B38F6087BB08956623DC
:1008900089F0813049F0813028F0823039F083309E
:1008A000C9F406C0C09A0895C19A0895C29A0895DD
:1008B000C39A0895813049F0813028F0823039F0B0
:1008C000833041F406C0C0980895C1980895C29835
:1008D0000895C3980895813051F0813030F082300E
:1008E00059F0833089F080E0089588B30BC088B355
:1008F00090E09695879506C088B390E09695879589
:10090000969587958170089588B390E023E0969539
:1009100087952A95E1F7817008958091B2008160F2
:100920008093B2008FEE86B9BC9A08952FB7F894E1
:10093000E82FF0E0EE0FFF1FEA56FF4F8081918114
:100940002FBF08952FB7F8948091B0009091B10017
:100950002FBF089580919500909195008917E1F33C
:100960000895823049F4809194006623C9F0826032
:1009700080939400A29A08958330A9F4662369F0C5
:1009800080919400836080939400A39A06C0809124
:1009900094008C7F8093940008956623C1F308959A
:1009A0008D7F80939400089508951F920F920FB643
:1009B0000F9211242F933F934F935F936F937F93E5
:1009C0008F939F93AF93BF93EF93FF938091930087
:1009D00024B135B14091B0005091B100420F531F86
:1009E0005093B1004093B000863009F460C0873066
:1009F00098F48230B1F1833030F4882319F18130DA
:100A000009F079C024C0843009F43FC0909194006B
:100A1000853008F03FC02AC0893009F458C08A30B8
:100A200038F4873009F448C0883009F064C049C000
:100A30008B3009F456C08B3008F44EC08C3009F06E
:100A40005AC054C030939B0020939A0054C03093F6
:100A50009D0020939C009091940091FF4CC0AA9817
:100A60004AC0309397002093960045C03093AD0064
:100A70002093AC00292F30E091FDAA9A23703070AA
:100A800021153105C1F1AB9836C030939900209300
:100A9000980031C03093AF002093AE00292F30E092
:100AA000237030702115310531F1AB9A24C0309399
:100AB000A1002093A0001FC03093A3002093A200A8
:100AC0001AC03093A5002093A400C49814C030939A
:100AD0009F0020939E000FC03093A7002093A60094
:100AE0000AC03093A9002093A80005C03093AB0042
:100AF0002093AA00C49A8F5F809393008D3058F0A2
:100B000010929300CA01880F991F57FD0196909388
:100B1000B1008093B00080919300863081F18730DE
:100B200070F4823009F1833028F48823C1F08130D9
:100B300051F518C08430E9F08530F8F418C08930D8
:100B4000E1F08A3028F48730E1F08830E1F413C016
:100B50008B30B9F08B3098F08C30A9F405C083E469
:100B600087B913C080E401C082E487B915C081E46D
:100B7000FCCF83E4FACF8EE5F8CF85E4F6CF86E4A8
:100B8000F4CF87E4F2CF882339F40E94D404809113
:100B900095008F5F80939500FF91EF91BF91AF918A
:100BA0009F918F917F916F915F914F913F912F9185
:100BB0000F900FBE0F901F90189584E00E9496042E
:100BC000BC0180E093EC0E946B0649E150E0649F19
:100BD0009001659F300D749F300D1124C901089557
:100BE0000F931F93082F162F81E061E00E944704A6
:100BF00082E061E00E94470480E061E00E944704D7
:100C000083E061E00E94470427E731E008C088EEF6
:100C100093E0F9013197F1F70197D9F701500023DB
:100C2000B1F781E060E00E94470482E060E00E944A
:100C3000470480E060E00E94470483E060E00E9497
:100C4000470427E731E008C088EE93E0F9013197C7
:100C5000F1F70197D9F711501123B1F71F910F91B7
:100C60000895CF93DF93EC0184E00E949604C817A7
:100C7000D90770F587B38F6087BB0E94C802F894CC
:100C800081B38F7081BB81E061E00E94F00581E05B
:100C900061E00E94F00581E061E00E94F00583E0E0
:100CA00061E00E94F00583E061E00E94F00583E0CE
:100CB00061E00E94F00581E061E00E94F00581E0C2
:100CC00061E00E94F00581E063E00E94F005DBCF67
:100CD000DF91CF910895AA1BBB1B51E107C0AA1F4A
:100CE000BB1FA617B70710F0A61BB70B881F991FCD
:100CF0005A95A9F780959095BC01CD01089597FB71
:100D0000092E07260AD077FD04D0E5DF06D00020A3
:100D10001AF4709561957F4F0895F6F79095819537
:100D20009F4F0895A1E21A2EAA1BBB1BFD010DC007
:100D3000AA1FBB1FEE1FFF1FA217B307E407F5078B
:100D400020F0A21BB30BE40BF50B661F771F881F67
:100D5000991F1A9469F760957095809590959B01FD
:0C0D6000AC01BD01CF010895F894FFCF55
:0C0D6C0001FC0000FF0301FC0000FF037D
:00000001FF
